:020000040801F1
:1000000000000220891B01088509010889090108EF
:100010008D090108910901089509010800000000F7
:100020000000000000000000000000009909010825
:100030009D09010800000000A1090108A5090108A7
:10004000D91B0108D91B0108D91B0108D91B0108BC
:10005000D91B0108D91B0108D91B0108D91B0108AC
:10006000D91B0108D91B0108D91B0108D91B01089C
:10007000D91B0108D91B0108D91B0108D91B01088C
:10008000D91B0108D91B0108D91B0108D91B01087C
:10009000D91B0108D91B0108D91B0108D91B01086C
:1000A000D91B0108D91B0108D91B0108D91B01085C
:1000B000D91B0108D91B0108D91B0108D91B01084C
:1000C000D91B0108D91B0108D91B0108D91B01083C
:1000D000D91B0108B5090108C1090108D91B01088C
:1000E000D91B0108D91B0108D91B0108D91B01081C
:1000F000D91B0108D91B0108D91B0108D91B01080C
:10010000D91B0108D91B0108D91B0108D91B0108FB
:10011000CD090108D91B0108D91B0108D91B010809
:10012000D91B0108D91B0108D91B0108D91B0108DB
:10013000D91B0108D91B0108D91B0108D91B0108CB
:10014000D91B0108D91B0108D91B0108D91B0108BB
:10015000D91B0108D91B0108D91B0108D91B0108AB
:10016000D91B0108D91B0108D91B0108D91B01089B
:10017000D91B0108D91B0108D91B01080000000088
:08018000D91B0108D91B01087D
:10018800044B05481B1A062B02D9044B03B1184728
:10019800704700BF2B00002028000020000000004E
:1001A80005490648091A891001EBD171491002D096
:1001B800034B03B11847704728000020280000208F
:1001C8000000000010B5064C237843B9FFF7D8FFAC
:1001D800044B13B10448AFF300800123237010BD12
:1001E8002800002000000000DC1B010808B5084BAF
:1001F8001BB108490848AFF300800848036813B9E1
:10020800BDE80840CCE7064B002BF9D09847F7E744
:10021800000000002C000020DC1B01082800002042
:100228000000000070B50F4E0F4D761BB61018BFBA
:10023800002405D0013455F8043B9847A642F9D16B
:100248000A4E0B4D761B01F0C5FCB61018BF0024F2
:1002580006D0013455F8043B9847A642F9D170BD41
:1002680070BD00BF041C0108041C0108081C01081B
:10027800041C010870B4860746D0541E002A41D0D9
:10028800CAB2034602E014F1FF343BD303F8012B52
:100298009D07F8D1032C2ED9CDB245EA05250F2CA0
:1002A80045EA054519D903F110022646103E0F2EDE
:1002B80042F8105C42F80C5C42F8085C42F8045CB6
:1002C80002F11002F2D8A4F1100222F00F0204F099
:1002D8000F041032032C13440DD91E462246043A4B
:1002E800032A46F8045BFAD8221F22F003020432DC
:1002F800134404F003042CB1C9B21C4403F8011BD5
:100308009C42FBD170BC704714460346C2E700BF4D
:10031800F0B595B008A830220021FFF7ABFF002404
:100328001D4A019404940394059406940794116C4F
:100338001A4B41F080511164126C02F08052019204
:10034800019A02941A6842F480421A601B680F945A
:1003580003F48043029301230225082148220B93CA
:1003680008A803231026109111921393029F089551
:100378000E9512950C9600F00BFF0F224FF4805348
:1003880003A829460495059407940392069301F05F
:10039800F5F815B0F0BD00BF00380240007000400D
:1003A80010B5064C00222046012101F0EBFA01228B
:1003B80020461146BDE8104001F0E4BA00040240AE
:1003C80070B5124D002401E0C92C1CD0012128462B
:1003D80001F0D2FAE3B201340028F5D1C82B12D0CB
:1003E8000A4E044601E0F12C0DD00121304601F0FF
:1003F800C3FAE5B201340028F5D0A5F1F000B0FA4F
:1004080080F0400970BD012070BD00BF00040240AB
:1004180010B5094C00222046012101F0B3FA01224F
:100428001146204601F0AEFA2046012101F0A4FA57
:10043800003018BF012010BD0004024038B5084D37
:10044800082400220121284601F09CFA01221146C5
:10045800284601F097FA631E13F0FF04F1D138BD66
:100468000004024008B5FFF79BFFFFF7A9FFCC2067
:10047800FFF7E4FF4420BDE80840FFF7DFBF00BFF7
:1004880070B582B0FFF7EEFFFFF78AFFFFF798FF1E
:10049800CC20FFF7D3FFBE20FFF7D0FF08240025AC
:1004A800FFF7B6FF6D08631E45EAC01513F0FF0499
:1004B800EDB2F5D10826FFF7ABFF6408731E44EAD6
:1004C800C01413F0FF06E4B2F5D1072C12D805EBDF
:1004D800042424B207EE904AF8EEE77AB6EE047ADE
:1004E80067EE877AFDEEE77ACDED017ABDF9040073
:1004F80002B070BD2302ED4383F47F4353FA85F3C2
:100508001BB207EE903AF8EEE77AB6EE047A67EE99
:10051800877AFDEEE77A17EE900A404200B202B001
:1005280070BD00BF474B484A484C80B59A6001F0FF
:10053800C9FAFFF7EDFE00F0A5F800F079F900F030
:100548003FF900F059F90A2305224149414800F0D2
:100558004BFC4FF47A7001F0DDFA0A2305223E497C
:100568003C4800F041FC21464FF4FA631422394814
:1005780000F096FC0A2314222146384800F034FC87
:10058800A37C5A1E012A56D9052B05D10A230B2212
:100598003349324800F028FC324D334CDFF8D8801C
:1005A800324FDFF8D890324EB3EE008AFFF768FF7B
:1005B800288042F2107001F0ADFAD4ED007AF4EE22
:1005C800C87AF1EE10FAF1D5404600224FF4806166
:1005D80001F0D8F9404600224FF4807101F0D2F9B9
:1005E800384600224FF4004101F0CCF93846002289
:1005F8004FF4005101F0C6F9384600224FF400616B
:1006080001F0C0F9484600224FF4004101F0BAF960
:10061800304600224FF4004101F0B4F93046002280
:100628004FF4005101F0AEF900224FF4006130465A
:1006380001F0A8F9B8E70A2307220E49074800F095
:10064800D3FBA9E700ED00E00000010854000020FA
:1006580008000020EC00002000000020AC00002072
:10066800180000204800002044000020000C024030
:100678000010024010000020000002400004024068
:10068800704700BF2DE9F0438BB00024464B00941F
:100698001A6B464DDFF82091DFF82081444F454E14
:1006A80042F001021A631A6B02F001020092009AEA
:1006B80001941A6B42F010021A631A6B02F01002CE
:1006C8000192019A02941A6B42F002021A631A6BA1
:1006D80002F002020292029A03941A6B42F0080294
:1006E8001A631A6B02F008020392039A04941A6BB5
:1006F80042F004021A631B6B03F0040304932846B8
:1007080001224FF47841049B01F03CF9484601224C
:100718004FF4404101F036F9404601224FF47C4144
:1007280001F030F9384601224FF4007101F02AF93E
:10073800012230464FF47C5101F024F9284605A9DE
:1007480001254FF47843059307940894069500F023
:10075800FDFF484605A94FF44043059306950794C5
:10076800089400F0F3FF404605A94FF47C43059335
:1007780006950794089400F0E9FF384605A94FF458
:100788000073059306950794089400F0DFFF4FF473
:100798007C5305A93046069507940894059300F004
:1007A800D5FF0BB0BDE8F0830038024000100240CE
:1007B800000802400000024000040240000C024011
:1007C8000B4B0C4A10B50C211A604FF4E13400228F
:1007D80018465C6059619A60DA601A619A61DA6158
:1007E80000F0D2FA00B910BDBDE81040FFF748BFCD
:1007F800AC000020004C00400B4B0C4A10B50C21FB
:100808001A604FF4E134002218465C6059619A601E
:10081800DA601A619A61DA6100F0B6FA00B910BDBF
:10082800BDE81040FFF72CBF6C000020001001400D
:100838000B4B0C4A10B50C211A604FF416440022D9
:1008480018465C6059619A60DA601A619A61DA61E7
:1008580000F09AFA00B910BDBDE81040FFF710BFCC
:10086800EC00002000440040F0B503683C4A934285
:1008780089B02BD03B4A93424DD03B4A934201D09A
:1008880009B0F0BD0024394B0294196C384841F482
:10089800003119641B6C03F400330293032207230D
:1008A80003A9602702260125DDF808E006920793D0
:1008B80003970496059500F049FF22462146262015
:1008C80001F088F8262001F0BBF8D9E70024274B6F
:1008D8000094196C274841F4002119641B6C03F437
:1008E800002300930322082303A94FF4406702263C
:1008F8000125DDF800E00692079303970496059515
:1009080000F024FF22462146342001F063F8342009
:1009180001F096F8B4E70024144B0194596C16487A
:1009280041F0100159645B6C03F01003019303223A
:10093800072303A9C02702260125DDF804E0069253
:10094800079303970496059500F000FF2246214679
:10095800252001F03FF8252001F072F890E700BF4C
:10096800004C0040001001400044004000380240A4
:10097800000C02400008024000040240704700BF1B
:10098800FEE700BFFEE700BFFEE700BFFEE700BFCF
:10099800704700BF704700BF704700BF08B501F03F
:1009A800ABF8BDE8084001F073B800BF014800F09B
:1009B80021BB00BF6C000020014800F01BBB00BF3A
:1009C800EC000020014800F015BB00BFAC0000207F
:1009D80008B5032000F0ECFF002211466FF00B0071
:1009E80000F0F8FF002211466FF00A0000F0F2FF55
:1009F800002211466FF0090000F0ECFF00221146BA
:100A08006FF0040000F0E6FF002211466FF00300CB
:100A180000F0E0FF002211466FF0010000F0DAFF5D
:100A2800002211464FF0FF30BDE8084000F0D2BF69
:100A38002DE9F047046822698246C068DAF81C107C
:100A4800DAF80830DAF81060DAF8145022F4405274
:100A580002432261E268DAF81800334322F41642AE
:100A68002B4322F00C020B431343E360636923F426
:100A780040730343B1F5004F6361AB4B61D09C42B7
:100A880000F0018103F580639C4200F0FC8000F0D7
:100A98002DFEA64FDAF8043000EB800000EB800052
:100AA8009B00B0FBF3F3A7FB03235B091D0100F0D8
:100AB8001DFEDAF8043000EB80009B0000EB80009C
:100AC800B0FBF3F600F012FEDAF8042000EB800029
:100AD800930000EB8000B0FBF3F3A7FB03234FF078
:100AE80064095B0909FB13631B013233A7FB03236A
:100AF8005B0903F0F00600F0F9FDDAF8042000EBDA
:100B08008000930000EB8000B0FBF3F800F0EEFDEE
:100B1800DAF8043000EB80009B0000EB8000B0FBAB
:100B2800F3F0A7FB0030400909FB10831B013233A7
:100B3800A7FB0323C3F3431333432B44A360BDE84C
:100B4800F0879C425DD003F580639C4259D000F049
:100B5800CDFD764FDAF8043000EB800000EB800022
:100B68005B00B0FBF3F3A7FB03235B091E0100F056
:100B7800BDFDDAF8043000EB80005B0000EB80007C
:100B8800B0FBF3F500F0B2FDDAF8042000EB8000CA
:100B9800530000EB8000B0FBF3F3A7FB03235B09D2
:100BA8004FF0640909FB1353DB003233A7FB03231F
:100BB8001B0903F4F87500F099FDDAF8042000EB3E
:100BC800800000EB80005300B0FBF3F800F08EFDCE
:100BD800DAF8043000EB800000EB80005B00B0FB2B
:100BE800F3F3A7FB03235B0909FB1383DB00323311
:100BF800A7FB0323C3F3421333442B44A360BDE88C
:100C0800F08700F08BFD494FDAF8043000EB8000E4
:100C180000EB80005B00B0FBF3F3A7FB03235B0949
:100C28001E0100F07BFDDAF8043000EB80005B0069
:100C380000EB8000B0FBF3F500F070FDDAF804205B
:100C480000EB8000530000EB8000B0FBF3F3A7FB40
:100C580003234FF064095B0909FB1353DB003233AC
:100C6800A7FB03231B0903F4F87500F057FDDAF816
:100C7800042000EB8000530000EB8000B0FBF3F889
:100C880000F04CFDA4E700F049FD284FDAF80430E5
:100C980000EB800000EB80009B00B0FBF3F3A7FBA8
:100CA80003235B091D0100F039FDDAF8043000EB7D
:100CB80080009B0000EB8000B0FBF3F600F02EFDF7
:100CC800DAF8042000EB8000930000EB8000B0FB12
:100CD800F3F3A7FB03234FF064095B0909FB1363D4
:100CE8001B013233A7FB03235B0903F0F00600F076
:100CF80015FDDAF8042000EB8000930000EB80007B
:100D0800B0FBF3F800F00AFDDAF8043000EB8000DD
:100D180000EB80009B00B0FBF3F3A7FB03235B0908
:100D280009FB138302E700BF001001401F85EB5148
:100D38002DE9F04107460E4690461D463C6801E005
:100D48006B1C06D1206836EA0003F9D10020BDE803
:100D5800F08135B100F0D8FEA0EB08008542EDD255
:100D68003C68E36823F4D073E3606369202223F0CE
:100D7800010300216361032087F8392087F83810C0
:100D880087F83A20BDE8F08160B338B590F839307B
:100D9800044603F0FF0203B32268242384F83930A1
:100DA800D36823F40053D3602046FFF741FE23683D
:100DB8001A6922F490421A615A6922F02A025A6189
:100DC800DA680025202142F40052DA602846E563FB
:100DD80084F8391084F83A1038BD80F83820FFF7C5
:100DE80043FDD9E7012070472DE9F0430F4690F8FD
:100DF8003910202983B003D0022003B0BDE8F08366
:100E0800002F3ED0002A3CD0984690F83830012B6D
:100E18000446F1D0002001212123E06384F8381032
:100E280084F83930019200F06FFE019AA28481465D
:100E3800E28406E0FFF77CFF28BB23683A785A6013
:100E48000137E58CADB243464A4680212046E5B1DC
:100E5800E58CA668013DADB2B6F5805FE584E9D1C1
:100E680043464A4680212046FFF762FF58B93B882F
:100E780021682269C3F308034B60002AE0D10237D6
:100E8800DFE70120B9E70320B7E74021FFF750FF6C
:100E98000028F8D1202384F8380084F83930ACE7EA
:100EA8002DE9F0430E4690F83A10202983B003D07C
:100EB800022003B0BDE8F08376B36AB3984690F891
:100EC8003830012B0446F3D0002001212223E063AF
:100ED80084F8381084F83A30019200F015FE019A2F
:100EE800A2858146E285E58DADB243464A4620217A
:100EF800204685B3E58DA768013DADB2B7F5805FA3
:100F0800E58512D0FFF714FF58BB236933B923686E
:100F18005B6833700136E6E70120CAE723685B683F
:100F280003F07F0333700136DDE743464A4620214C
:100F38002046FFF7FDFEA0B9236933B923685B6833
:100F4800C3F3080326F8023BCDE723685B68DBB2EE
:100F580026F8013BC7E784F83850284684F83A1049
:100F6800A7E70320A5E700BF704700BF704700BF91
:100F78008368B3F5805F28D0036973B10368826A18
:100F88005B68511C03F07F0381621370C38D013BC2
:100F98009BB2C38543B100207047836A0268591C1D
:100FA800526881621A70F1E70268D16821F4907181
:100FB80010B5D1605169202421F00101516180F8F8
:100FC8003A40FFF7D3FF002010BD0269836A3AB99F
:100FD80002685268C2F3080223F8022B8362D5E73D
:100FE80002685268D2B223F8012B8362CEE700BFB1
:100FF800704700BF03681A6870B51607DD6859693D
:10100800044649D011F0010152D0D60705D5E805AC
:1010180003D5E06B40F00100E06356077AD500295C
:1010280000F08480E16B900741F00201E16376D51E
:10103800E16B41F00401E163110772D4E16B00290F
:1010480029D0910605D5AA0603D594F83A20222A74
:101058007CD05D69E16B0E0702D415F040057AD0AB
:10106800DA6822F49072DA605A69202122F00102CB
:101078005A6184F83A105A6955065ED55A69606B08
:1010880022F040025A61002857D03B4B036500F01C
:101098007DFC002855D170BD96060CD5A9060AD549
:1010A80090F83A30222BF6D1BDE87040FFF760BFC8
:1010B80015F4907FA9D110060ED45606EBD56D060F
:1010C800E9D5DA68202122F04002DA60204684F867
:1010D8003910FFF749FF70BD2906EED594F839207D
:1010E800212AD8D1A268B2F5805F226A38D0511C73
:1010F800216212785A60E28C013A92B2E284002AA4
:10110800C9D1DA6822F08002DA60DA6842F0400277
:10111800DA6070BD96070BD5002989D18EE71107D3
:101128008CD5E16B41F00801E16387E7900785D42E
:10113800100783D5002981D0F3E72046FFF758FF31
:1011480070BD606BBDE87040036D18472046FFF71F
:101158000FFF23687DE72046FFF74AFFE56370BD70
:1011680011882069C1F30801596010B9023222625E
:10117800C1E701322262BEE78511010808B5836B19
:101188000022DA851846DA84FFF732FF08BD00BF6F
:10119800F0B50368DD0783B004462FD5A3498A68F4
:1011A80002F00C02042A00F0F4808A6802F00C02B3
:1011B800082A00F0EA806368B3F5803F00F02C81CC
:1011C800B3F5A02F00F00081984D2A6822F48032F0
:1011D8002A602A6822F480222A60002B40F0FD80D1
:1011E80000F092FC064605E000F08EFC801B6428A7
:1011F80000F2AA802B689B03F6D423689F072DD59D
:101208008A4A916811F00C0F00F0A580916801F0EE
:101218000C01082900F09B80E368002B00F0EB80AC
:10122800834B824D01221A6000F06EFC064605E0F1
:1012380000F06AFC801B022800F286802B68980761
:10124800F6D52968F82292FAA2F22369B2FA82F254
:1012580021F0F80193400B432B6023681A0720D430
:10126800590734D4A369CBB1704DAA6802F00C02B7
:10127800082A77D0022B6F4B4FF000021A6000F05B
:10128800D18000F041FC2C46054604E000F03CFC0F
:10129800401B022858D823689B01F7D4002003B0CC
:1012A800F0BD6369002B60D0634B604D01221A606A
:1012B80000F02AFC064604E000F026FC801B022809
:1012C80042D86B6F9F07F7D523685907CAD5574B84
:1012D8005A4D002201921A6C42F080521A641B6C1B
:1012E80003F080530193019B2B6843F480732B60B8
:1012F80000F00AFC064604E000F006FC801B022809
:1013080022D82B68DA05F7D5A368012B00F0F18005
:10131800052B00F0D580454D2A6F22F001022A677F
:101328002A6F22F004022A67002B40F0D28000F0D6
:10133800EBFB41F2883607462B6F980792D500F0F1
:10134800E3FBC01BB042F7D9032003B0F0BD5268DD
:1013580056023FF561AF354A1268950723D5E26812
:10136800012A20D0012003B0F0BD334A2F4D13606D
:1013780000F0CAFB064604E000F0C6FB801B02280A
:10138800E2D86B6F9807F7D49EE74A6850027FF55A
:1013980012AF264A126891037FF530AF6268002ABF
:1013A8007FF42CAFDEE7214DF821286891FAA1F1EE
:1013B8002269B1FA81F120F0F8008A4002432A60DC
:1013C8001A077FF54DAF6CE7184B1A6842F4802274
:1013D8001A601A6842F480321A6000F095FB134DC7
:1013E800064604E000F090FB801B6428ACD82B680C
:1013F8009A03F7D501E70E4A0C4D136000F084FB01
:10140800064604E000F080FB801B02289CD82B686D
:101418009907F7D4236821E7044A136843F4803313
:101428001360DAE700F070FB06460FE00038024070
:101438000000474260004742800E4742007000406B
:1014480000F062FB801B02283FF67EAF2B689901F3
:10145800F6D447F6C07696FAA6F64FF44032B6FAB6
:1014680086F692FAA2F24FF07061B2FA82F091FA1F
:10147800A1F1A26A676AE369D4F820E0E46A520835
:1014880043EA0E0307FA06F6013A8240B1FA81F1FF
:10149800334304FA01F11343194A1A4C0B4301214F
:1014A8006B60116000F030FB054605E000F02CFB96
:1014B800401B02283FF648AF23689A01F6D5EDE6AF
:1014C800104B1A6F42F004021A671A6F42F00102B9
:1014D8001A6700F019FB0B4D074641F288362B6F4F
:1014E8009B073FF5BFAE00F00FFBC01BB042F6D91B
:1014F8002AE7044A136F43F001031367E9E700BFC3
:101508006000474200380240194A936803F00C0310
:10151800042B2BD0082B27D15168536801F03F01C9
:1015280013F4800F536847F6C07292FAA2F0B0FA2B
:1015380080F003EA020323FA00F314BF0D480E48B3
:10154800B0FBF1F000FB03F0094B4FF440325B684D
:1015580092FAA2F2B2FA82F203F44033D340013392
:101568005B00B0FBF3F070470348704701487047D1
:101578000038024040787D010024F400574A13687F
:1015880003F00F038B4208D2CBB21370136803F039
:101598000F03994201D00120704703689A072DE98B
:1015A800F04106D54E4C8568A26822F0F0022A4325
:1015B800A260DF0706460C4626D54268012A00F0DD
:1015C8008780931E012B464B1B687BD9990728D52A
:1015D800434DAB6823F003031343AB6000F094FA68
:1015E8007368012B074641F288384FD0022B58D038
:1015F800032B05D160E000F087FAC01B404564D892
:10160800AB6813F00C0FF6D1344A136803F00F03DC
:101618009C4209D2E3B21370136803F00F039C4293
:1016280002D00120BDE8F08133685A0706D52C495D
:10163800F0688A6822F4E05202438A601B0707D5E3
:10164800274A3169936823F4604343EAC1039360EE
:10165800FFF75AFF224B0146F0229B6892FAA2F24A
:10166800B2FA82F203F0F003D3401E481E4AC35C6C
:10167800002021FA03F3136000F00EFA0020BDE801
:10168800F08100F041FAC01B40451ED8AB6803F05A
:101698000C03042BF5D1B7E700F036FAC01B404520
:1016A80013D8AB6803F00C03082BF5D1ACE700F0B6
:1016B8002BFAC01B404508D8AB6803F00C030C2B71
:1016C800F5D1A1E7980183D4ABE70320BDE8F08109
:1016D800034B1B689D033FF57BAFA2E7003C02402C
:1016E80000380240F41B010824000020084B4FF486
:1016F800E0529B6892FAA2F2B2FA82F203F4E05343
:10170800D3400449044ACB5C1068D840704700BFF6
:1017180000380240F41B010824000020084B4FF455
:1017280060429B6892FAA2F2B2FA82F203F4604332
:10173800D3400449044ACB5C1068D840704700BFC6
:1017480000380240F41B0108240000202DE9F04F66
:10175800D1F800C0DFF81482DFF814E283B0002566
:1017680003E00135102D00F09B800123AB4003EA14
:101778000C029342F5D14E6826F0100ABAF1020F16
:1017880000F091804FEA45090324D0F800B004FA2C
:1017980009F4E44306F003070BEA040B07FA09F718
:1017A8000AF1FF3A47EA0B07BAF1010F076040F266
:1017B800A080C7688B683C4003FA09F32343C360E1
:1017C800F300CED54FF00009CDF80490D8F8443096
:1017D80043F48043C8F84430D8F8444025F0030364
:1017E80003F1804304F4804403F59C33019405F02D
:1017F8000304019FD3F808A0A4000F27A7402AEAF2
:10180800070A544FB84222D007F58067B84200F063
:101818008380514FB84200F08480504FB84200F0A6
:1018280085804F4FB84200F086804E4FB84200F096
:1018380087804D4FB84200F08880DFF838914845DE
:101848000CBF4FF007094FF0080909FA04F94AEAF2
:1018580009079F60DEF80030D443F70354BF2340E4
:101868001343CEF80030DEF80430B70354BF2340EA
:101878001343CEF80430DEF80830F70254BF234093
:101888001343CEF80830DEF80C30B60205F1010536
:1018980054BF23401343102DCEF80C307FF465AFAE
:1018A80003B0BDE8F08F4FEAD50900EB890905F0D0
:1018B8000707D9F82040BF004FF00F0B0BFA07FBC2
:1018C80024EA0B0A0C69BC4044EA0A04C9F820401F
:1018D8004FEA45090324D0F800A004FA09F4E443C8
:1018E80006F003070AEA040A07FA09F747EA0A07AB
:1018F8000760876807EA040ACF6807FA09F747EA22
:101908000A078760D0F804A0C6F300172AEA030381
:10191800AF401F4347604CE74FF0010909FA04F94B
:1019280095E74FF0020909FA04F990E74FF0030927
:1019380009FA04F98BE74FF0040909FA04F986E774
:101948004FF0050909FA04F981E74FF0060909FA89
:1019580004F97CE70000024000080240000C024045
:1019680000100240001402400018024000380240F3
:10197800003C0140001C02400369194214BF0120C9
:101988000020704702B909048161704790F835302A
:10199800022B03D08023436501207047026805238A
:1019A80080F83530136823F0010313600020704776
:1019B800074AD3684FF6FF010B40000243F0BF63AC
:1019C80000F4E06043F400330343D360704700BF82
:1019D80000ED00E0184B70B4DC68C4F30224C4F1D5
:1019E8000706042E04F1040328BF0426062B17D982
:1019F800033C0125A540013D2A400123B340013B9A
:101A08001940A140002841EA02010CDB00F16040C6
:101A180000F561400901C9B280F8001370BC704735
:101A280000221446E9E7054B00F00F0009010344C2
:101A3800C9B2197670BC704700ED00E0FCEC00E01C
:101A480000F01F0101234009024A8B4042F8203070
:101A5800704700BF00E100E00138B0F1807F0ED28E
:101A6800084B10B4084C5860F02084F8230000227A
:101A7800072110469A6019605DF8044B70470120F1
:101A8800704700BF10E000E000ED00E0704700BFC5
:101A980008B5FFF7FBFF08BD084B094A1B6810B5DE
:101AA800A2FB032304469809FFF7D6FF214600222C
:101AB8004FF0FF30FFF78EFF002010BD24000020FC
:101AC800D34D621008B50B4B1A6842F400721A60C5
:101AD8001A6842F480621A601A6842F480721A60C6
:101AE8000320FFF765FF0020FFF7D6FFFEF770FF22
:101AF800002008BD003C0240024A1368013313600D
:101B0800704700BF2C010020014B1868704700BFC8
:101B18002C01002010B582B00190FFF7F5FF0446B4
:101B2800FFF7F2FF019B001B9842F9D302B010BDEA
:101B38001049114BD1F8882042F4700210B4C1F852
:101B480088201A680D4C002042F001021A60986043
:101B58001A6822F0847222F480321A605C601A6873
:101B68004FF0006422F480221A60D8608C605DF81F
:101B7800044B704700ED00E00038024010300024AC
:101B8800DFF834D0002103E00C4B5B58435004319C
:101B98000B480C4B42189A42F6D30B4A02E000233A
:101BA80042F8043B094B9A42F9D3FFF7C1FFFEF70D
:101BB80039FBFEF7B7FC7047000002200C1C010837
:101BC800000000202800002028000020300100200C
:101BD800FEE70000F8B500BFF8BC08BC9E46704799
:0C1BE800F8B500BFF8BC08BC9E46704772
:101BF40000000000010203040102030406070809AF
:041C0400F5010108DD
:041C0800CD01010801
:101C0C00FE00010001000000FE00020002000000C6
:101C1C00636F6E6E656374006E6F7420636F6E6EAF
:081C2C00656374000024F4005C
:0400000508011B894A
:00000001FF
